:030000000219FDE5
:03000B000200A848
:03002B000201547B
:03005B000202DDC1
:030073000202CABC
:1000800002030406080C10182030406080040608A3
:100090000C10182030406080A0C00003070F1F051F
:1000A000050D050205030302C2AFC0D0C0E0206207
:1000B00014E5256009E473E525F4F58AD262D0E001
:1000C000D0D0D2AF3285268AC262E526F46029D02C
:1000D000E0D0D0D290D291D292D2AF32D290D291FF
:1000E000D292206F0C206609740AD5E0FDE57B42B0
:1000F00090D0E0D0D0D2AF32758A00C28DD26201EA
:10010000F101B7306805206602C29001B73068057A
:10011000206602C29101B7306805206602C29201D2
:10012000B7C29330680A2066077408D5E0FDC29014
:1001300001B7C29430680A2066077408D5E0FDC292
:100140009101B7C29530680A2066077408D5E0FDB2
:10015000C29201B7C2AFC2AD53E6EFC0D0C0E0D289
:10016000D3D2AFC2CEE52A6007207449152A21B543
:100170007800790020742EE580307E01F430E702AB
:1001800078FF53DACF207E0343DA20307E0343DA50
:1001900010C2D8C271E580307E01F430E70279FFE9
:1001A000C3E89970CB306103752A18207403752A4F
:1001B00018885CD27020740DE52B6004152B21C5C6
:1001C00043DA01C2D82070024138A85C206102C223
:1001D00070207431C3E894F0400374F0F8E8C4541C
:1001E0000F28F87984B703024105C313C31387218D
:1001F000200802C313200A06C3C898F8410528F84E
:10020000500374FFF8C3E895655003E565F888224C
:10021000E52D54066022206B1FE536C333C333F847
:10022000E564C313C313F9C3952240028922E8256C
:1002300022F52250037522FF852224A824C3E52439
:1002400095614002A8618825E5667002417CC3E89B
:10025000AA669A5003E8FAE4F9EAC333FBE568F4C6
:100260005B29400D2567F8E56760021567400B4183
:100270007C0AC3E5679A5002056778FF8826C3E5C4
:100280002594404002D26420CF0AD0E0D0D043E68B
:1002900010D2AD32C2CF053A7801E52A600530743C
:1002A00002152AC3E55C94014005755F0041C075E5
:1002B0006000756900E55F2401F55F5003755FFF1D
:1002C000D0E0D0D043E610D2AD32C2AF53E67F7556
:1002D00092FA7593FFC260759104D2AF32C2AF53E8
:1002E000E6EFC2ADC0D0C0E0C0F0D2D3D2AFA8FB21
:1002F000A9FCC2D8307102614453DACF207E034397
:10030000DA10307E0343DA20D271E580307E01F4CA
:1003100020E702611B88278928A17153DACF207E4C
:100320000343DA20307E0343DA10C2D8C27130743E
:1003300002A15D7800E580307E01F430E702A15D26
:10034000885CA14553DACF207E0343DA20307E0358
:1003500043DA10C271206102811D53DACF207E037F
:1003600043DA10307E0343DA20C2D8D2718857892D
:1003700058C3E89555F8E99556F97B007E087A0050
:10038000C3E8948CE994005005755B00810F8821C7
:1003900078A2E6A8216055C3E894C8E99400500803
:1003A000E4D2E4FB7A0A61EAC3E89468E994015074
:1003B00008E4D2E3FB7A0F61EAC3E894D0E994023F
:1003C0005008E4D2E2FB7A1E61EAC3E894A0E99403
:1003D000055008E4D2E1FB7A3C61EAC3E89498E96D
:1003E00094085008E4D2E0FB7A787E00C3E895597F
:1003F000FCE9955AFD30E70AECF42401FCEDF434F5
:1004000000FD755B00C3EC9AED9E5003755B01889F
:1004100059895A8557558558567802A145C3E8959C
:1004200027F8E99528F9307C02A129307B02A1291F
:10043000307A02A1222075028140E9FDE8FC815F4B
:10044000E9C313F9E813F8307902A122E9C313F9DB
:10045000E813F8307802A122E9C313FDE813FC2069
:10046000612CC3EC941CED940240028176ED701E69
:0F047000C3EC94C850180529E52970021529C35B
:10047F00E529940A5002A15D755C00D270A15DE57B
:10048F0029600215297888E6F97400207F0878968C
:10049F00B90302789EE624FAFEE43400FFC3EC9E13
:1004AF00FCED9FFD9208B90310A2085007207609B2
:1004BF00D27681C8307602C276A2085016B9030DE3
:1004CF00ECF42401FCEDF43400FD0204E278007931
:1004DF0000A129B90315EC33FCED33FDC3EC940AED
:1004EF00FCED9400FD50047C007D00C3EC94FFED07
:1004FF009400400678FF7900A129EC8572F0A4C51D
:10050F00F0A2F733F87900400302054578FF790030
:10051F00020545E9C313F9E813F8307C0EE96002D0
:10052F0078FFC3E81338F8E43400F9C3E894FFE91F
:10053F009400400278FF885CD270206102A15D7444
:10054F001FF4552F4BF52FC274EB7002D274752A1E
:10055F0018307403752A0A306102A1712074035395
:10056F00DAFE207403752B06D0F0D0E0D0D0D2ADD8
:10057F0043E6103279010205A179030205A1790A38
:10058F000205A1791E0205A179640205A179C802AD
:10059F0005A17817E4D5E0FDD8FAD9F6227A147BB5
:1005AF00780205C87A107B8C0205C87A0D7BB402DD
:1005BF0005C87A0B7BC80205C87902E4C294D5E05E
:1005CF00FDC291D5E0FDD291D5E0FDD294D5E0FDED
:1005DF00E920E002C29030E002C292E573D5E0FD5F
:1005EF00E920E002D29030E002D2927496D5E0FD7D
:1005FF00D9C9EAF8D5E0FDD8FBDBBEC29422C37C93
:10060F00007D0075F00005F0EA33FAEB33FB50F68E
:10061F00EB13FBEA13FAC3E9FFE8FEE89AF8E99B4C
:10062F00F95004EFF9EEF8B3EC33FCED33FDD5F0F0
:10063F00DFEDF9ECF822E889F08A20D2D4F8A9F09E
:10064F007B0030F70B7BFFF42401F8E9F43400F959
:10065F00E88520F0A4ADF0F8E98520F0A4AFF0FE16
:10066F00ED2EF974003FFA7C04C3EA13FAE913F98B
:10067F00E813F8DCF48BF030F70AE8F42401F8E91A
:10068F00F43400F9E889F0C2D4F8A9F02222C3E5C6
:10069F004113F9E54013F8C3E54498F8E54599F996
:1006AF00500CC3E89480E994FF40160206D4C3E8C7
:1006BF00947FE9940050030206D4787F79000206F4
:1006CF00D4788079FF8849894A22E5492546F8E59B
:1006DF004A3547F9854A20E4300701F43548FA30A6
:1006EF00E709C3EA94F04015020712C3EA940F50CA
:1006FF000302071278FF79FF7A0F02071278007949
:10070F00007AF0C3E5249561500AC3740195245013
:10071F000B020730E54A20E70E020730E54A30E7C3
:10072F0006884689478A482278A5E6FAC3E5493301
:10073F00F8E54A33F9D145E930E70BC3E89480E98E
:10074F0094FF4013E16AC3E8947FE994005002E1FB
:10075F006A787F7900E16A788079FFE820E715C32E
:10076F00E52398F84009C3E8940140030207917804
:10077F0001020791E8F424012523F84003020791B1
:10078F0078FF884B2278A6E6FAA847A948D145E911
:10079F0030E70CC3E89401E994FF40160207C5C384
:1007AF00E894FFE9940050030207C578FF7900022F
:1007BF0007C5780179FFE920E715C3E54B98F840A5
:1007CF0009C3E8940140030207EC78010207ECE843
:1007DF00F42401254BF840030207EC78FF8824220C
:1007EF0078FFC26420693D206A12D264C3E5419448
:1007FF000A4009C3E52594405002C26479A1E7601D
:10080F0023E541601F74FF8541F0848539F0306A1C
:10081F000375F005A4F8C5F0600278FFC3E895648E
:10082F005002A864886322C3E5409440E5419401D7
:10083F00E5635003140147046002F5632202084F79
:10084F002275E890227883E6FFE5E820ECF7A8BD53
:10085F00A9BE0570C3E57094084052757000E9FA9F
:0F086F0079A0E76044EA7007E571601B02088A10
:10087E00C3E895716010E5715006600C140208967D
:10088E000460F9020896E571F571C3946D401B750D
:10089E0061C0C394044013756180C39404400B750A
:1008AE006140C39404400375610075BB0622E56187
:1008BE00F460020561E570B4070375BB1022743253
:1008CE0079A787F0A4C5F0A2F733F8C3E895614085
:1008DE0002A861882288248825882688642275408B
:1008EE00007541F022C2AF75C820A8CCA9CDAA3A96
:1008FE0030CF010A75C824D2AFAB3BAC3C883B89E4
:10090E003CC3E89BF8E99C206908F930670221FF97
:10091E00215CAD3D8A3DF9EA9DFA600478FF79FFCE
:10092E00AE3EAF3F8B3E8C3FA83BA93CC3E89EF842
:10093E00E99FF9C3E54113FBE54013FAE82AF540B8
:10094E00E93BF54150067540FF7541FF21A6AA40CF
:10095E00AB41AC40AD417E047F02C3EB9404400238
:10096E001E1FC3EB940840021E1FC3ED13FDEC13B4
:10097E00FCDEF7C3EA9CFAEB9DFBEF6009C3E913BB
:10098E00F9E813F8DFF7EA28FAEB39FB8A408B41D6
:10099E0050067BFF8B408B41C3EB94025002D26713
:1009AE003069047F0321D17892E6FFC3E537948244
:1009BE0040110FC3E53794A040010FC3EF940640DA
:1009CE00027F057E02E541C4540FF9E541C454F09F
:1009DE00F8E540C4540F28F8C3E89EFAE99400FBEA
:1009EE004009C3EA9402EB940050047A02E4FB41FE
:1009FE004BAA40AB41EBC4FEEAC4540F4EFCC3EA13
:100A0E009CFAEB9400FBC3E813C313F8EA28FAEB45
:100A1E003400FB8A408B41C3EB94024002C26778DC
:100A2E0002EBC4FE7B00EAC4540F4EFAC3EA98FAF6
:100A3E004005C3940250027A027892E6FF306002BB
:100A4E00414B855192855293D26043E680C3E49A1E
:100A5E00F8E49BF930670241D7E8FAE9FBD3E913D2
:100A6E00FDE813FC88518952C3EF94036038EF20E0
:100A7E00E00DE82CF8E93DF9ECFAEDFB020AA0E8EE
:100A8E0028F8E939F9C3E82402F8E93400F97AFEC6
:100A9E007BFFC3EF9403400E8A538B54884D894ECF
:100AAE008C4F8D50610B885389548A4D8B4E8C4FD1
:100ABE008D503069127553F07554FF754FF07550A7
:100ACE00FF7551F07552FF610BE8FAD3E813FC88FD
:100ADE0051C3EF94036020EF20E007E82CF8ECFA06
:100AEE0041F7E8282402F87AFEC3EF940340088AFF
:100AFE0053884D8C4F610B88538A4D8C4FE568C3DC
:100B0E00335002646BF5683060026115753402D2A1
:100B1E006043E680E52D54066034A840A941C3E940
:100B2E0013F9E813F8C3E913F9E813F8306904E987
:100B3E002440F9C2AF53E67F759100C3E498F59453
:100B4E00E499F595759104D26043E680D2AF22D236
:100B5E0065754300752000306C03752040020B7CD8
:100B6E00D265754300752040306C03752000780106
:100B7E007901206720E52D54066002C2657914E5DF
:100B8E0041C313700104F8C3941440027814306901
:100B9E0004781B791B206010E543600C306903D587
:100BAE003404D26D811F711D0543E59BF45440B58D
:100BBE002002810930690908C3E89940011861A330
:100BCE0020650A08C3E8994002617C61A3C265C230
:100BDE00AF53E67F7591003067127594007595FEE0
:100BEE00759104D26043E680D2AF617CAE40AF41D6
:100BFE00C3E49EF594E49FF59561EEC3E53394014D
:100C0E005002617C306502617CD802811D61A3C2F5
:100C1E006DC2AF53E67F75910085539485549575DB
:100C2E009104854D92854E93D26043E680D2AFE516
:100C3E002D54066008206A020533020C5B306D0DE0
:100C4E00206C0A206507158115810214F1227800A7
:100C5E003064053065027801E53775F007A4F9E5D3
:0E0C6E00F028F5F0E9A2F013A2F113A2F213A0
:100C7C00F537C394785003753778C3E5379538400A
:100C8C0008D266D290D291D2923060028195854F73
:100C9C0092855093D26043E68022207D16C2AF75B8
:100CAC004202C294D293306202C292D2AF759F11AB
:100CBC00020E95C2AF754202C294D295306202C246
:100CCC0090D2AF759F11020E95307243207D20C2D9
:100CDC00AF754203900132757B10D292C29530628F
:100CEC0004C29181F3D294D2AF759F21020E95C2AA
:100CFC00AF754203900132757B10D290C293306273
:100D0C0004C291A113D294D2AF759F01020E95200B
:100D1C007D17C2AF75420390010DD292306202C2B0
:100D2C0091D2AF759F21020E95C2AF75420390010F
:100D3C000DD290306202C291D2AF759F01020E9516
:100D4C00207D16C2AF754204C293D295306202C2A6
:100D5C0091D2AF759F01020E95C2AF754204C29538
:100D6C00D293306202C291D2AF759F21020E9530A0
:100D7C007243207D20C2AF754205900121757B081E
:100D8C00D291C294306204C290A199D293D2AF7521
:100D9C009F11020E95C2AF754205900143757B20E1
:100DAC00D291C294306204C292A1B9D295D2AF75DD
:100DBC009F11020E95207D17C2AF7542059001035D
:100DCC00D291306202C290D2AF759F11020E95C2C1
:100DDC00AF754205900117D2913062EBC292D2AF3F
:100DEC00759F11020E95207D16C2AF754206C295F5
:100DFC00D294306202C290D2AF759F21020E95C27E
:100E0C00AF754206C293D294306202C292D2AF75D1
:100E1C009F01020E95307243207D20C2AF754201B6
:100E2C00900143757B20D290C293306204C292C170
:100E3C003FD295D2AF759F01020E95C2AF7542019C
:100E4C00900121757B08D292C295306204C290C188
:100E5C005FD293D2AF759F21020E95207D17C2AF42
:100E6C00754201900117D290306202C292D2AF75D6
:100E7C009F01020E95C2AF754201900103D29230D0
:100E8C006202C290D2AF759F21C266229001017599
:100E9C007B00D290D291D292C293C294C295C2627C
:100EAC0022788076FF0876FF0876FF0876FF0876B2
:100EBC00030876040876080876010876010876019E
:100ECC00788C76010876FF0876FF0876FF0876FFA7
:100EDC000876FF0876030876FF0876FF0876FF0889
:100EEC0076250876D00876FA0876FA08760408761D
:100EFC00FF08760108760008767A0876FF087601F6
:100F0C00087601087600087603087600227887E6D2
:100F1C00FFC2727888E6C394036008C27DE630E1B4
:100F2C0002D27DC27E7889E630E102D27EC3EF9494
:100F3C00026008758E01D273020F4C758E00C2735D
:100F4C00227880E6149000809378A5F67881E614D8
:100F5C009000809378A6F67886E61490008D9378AE
:100F6C00A7F67886E6F539C39402500375390278F2
:100F7C009CE67538FFB402037538A0B403037538CA
:100F8C008278A3E61490009A93F566D19822227881
:100F9C0096E6FA7897E6FB7888E6B40305C3EB94FB
:100FAC000EFB307F047A007BFFC3EB9AFCC3948268
:100FBC0050027C827572000572EC8572F0A4C3E558
:100FCC00F0947D40F222D27FF19B1205927A007B45
:100FDC00007C10120588E55C2AFA74003BFBDCF3FC
:100FEC007C04C3EB13FBEA13FADCF7FEC27FF19B24
:100FFC0022E5EF20E6037520000520903FFFE52059
:10100C00146006901DFF1460009304600375EF12CA
:10101C0053D9BF7581C043FF8012058375EF02431E
:10102C00B203E5B3240220E70DF521E5E320E00649
:10103C008521B343E301120E987580FF75A40075EA
:10104C00F19175D47F75900775A53F75F2FF75D535
:10105C000075A60175E241120E98E4F8F6D8FD75FC
:0F106C006801120EAD1215427898867375300127
:10107B00C2AF12059C1205AC1205921205B31205F4
:10108B00921205BA12059212165B12059C12059C60
:10109B00120597C2AF78FA79FA308707D9FBD8F7E0
:1010AB00021C00120F19120F4D120F9A120F9B7880
:1010BB00988673120E9875881075890275C82475F9
:1010CB00910475D84075A82275B80275E690759B8A
:1010DB0080759D0075D10E75BC5875BB0675BA1120
:1010EB0075E880120583D2AF12084C75360053DABF
:1010FB00CF207E0343DA20307E0343DA1043DA013C
:10110B00C2D8C27112059CD2617B037A0CE55B706D
:10111B00077A0CDB0302109E12059220700302105B
:10112B009EC270E55CC3940240E1E52F541F855EBF
:10113B005DF55EB55DD5DAD5C26153DACF207E039E
:10114B0043DA20307E0343DA10C2D8C27178A2E6AC
:10115B007008D274E52F54E0F52FC2757529001273
:10116B000597307409C3E529940A4002D27512051C
:10117B008878023074027800C3E55C9840F0C2AF07
:10118B001205AC1205AC1205ACD2AF12059C754C16
:10119B00007888E6B403024181120588788CE6C397
:1011AB0094015003021281E530C3940150030212E3
:1011BB0081207435C3E55C94FF5003021281C2AFEA
:1011CB001205C1D2AF120597C3E55C940150EFC273
:1011DB00AF1205AC12058D1205ACD2AF120597C339
:1011EB00E55C94FF40E90216E07F05D27F120F9B6E
:1011FB00120597C2AFC27F120F9BAE5CC3E55C9426
:10120B007FD2AF407B120583C2AF1205C1D2AFDFD5
:10121B00DA120FD2C3EE94057897F612059C1215CD
:10122B00841216637F0AD27F120F9B120597C2AFEF
:10123B00C27F120F9BAE5CC3E55C947FD2AF50E4D0
:10124B00120583C2AF1205AC12058D1205ACD2AFDD
:10125B00DFD4120FD2EE24037896F612059C1215EA
:10126B0084121692120597120F9BC3E55C94FF50E4
:10127B000221BC0216E0C3E55C954C4003855C4C37
:10128B0012059778017988E7B403027805C3E55C0A
:10129B00984002219CC2AF1205C11205C11205C1B3
:1012AB00D2AF12059C753000E4F531F5320531E50E
:1012BB0031F4703F0532789AE6781914601278325F
:1012CB0014600D787D14600878FA14600375320091
:1012DB00C3E53298401D120E9812058315327531F5
:1012EB000078998673C2AF1205C1D2AF7898867316
:1012FB0012059712058DE52A7005307402019E7850
:10130B00012074027806C3E55C9840A17888E6C397
:10131B0094036003120597E52A700302109EC2AF77
:10132B00120E98E4F522F523F524F525F526F5673D
:10133B00D2AF7885E6C333F565E4F544F545F5465C
:10134B00F547F548F570F52CF52DF53775700875E3
:10135B00BB10120583120850E5E820ECFBA8BDA9D1
:10136B00BEE97001F8887112085475700875BB10CE
:10137B00120F19C2AF7561FF1208CC85226185224D
:10138B0062852263D2AF7522017524017525017523
:10139B002601856069756A017888E6B40307C27D0A
:1013AB00307602D27DD268D269753300120DF212FB
:1013BB000E211208EC1208F31208EC1208F31208B3
:1013CB00EC120B6E12069C120C5C120CA61208F39C
:1013DB00120B5D306E0312069D2067031207EF3070
:1013EB006703120836120C5C120CD51208F3120BA1
:1013FB006E306E031206D9120C5C120D4C1208F3F0
:10140B00120B5D306E03120737120C5C120D7B1240
:10141B0008F3120B6E306E03120794120C5C120D54
:10142B00F21208F3120850120B5D120C5C120E2113
:10143B001208541208F330692F8564618564628544
:10144B006069756A0179187A0CC3E53399400CC24F
:10145B0069D26A8A357561FF021473C3E55C940126
:0E146B0040030213CC0214F9306A1D206C1AE3
:10147900E535147006C26AD26B61CCF535C3E55CFB
:10148900940140030213CC0214F97536007882796D
:10149900A4E760027803C3E55F985054307404E50B
:1014A9002A604D7888E6B40317207D0520760781E8
:1014B900C930760281C9206C07D26C856461810BC1
:1014C90078F0306C058564617820C3E54198500255
:1014D90061CC306C1BC26CC27D307602D27DD26A7F
:1014E90075351285646161CC0536E55C600281FC65
:1014F900753600C2AF120E987887E6FE7602120F93
:10150900197887EEF6E4F522F523F524F525F52675
:10151900F565752C00752D00D2AF120597120E983E
:1015290078A4E66006C290C291C292307409C3E5FC
:101539003694044002019E41B3901A0D7820121589
:10154900C6E520B45A0CA31215C6E520B4A50302BA
:101559001564120EAD121584021583901A03788052
:101569007B0A1215C6A308DBF9901A0F788C7B1930
:101579001215C6A308DBF9901A2822C2AF12160564
:101589001215DF901A00740E1215CBA374061215EA
:10159900CBA374151215CB901A0378807B0A121508
:1015A900CAA308DBF9901A0F788C7B191215CAA304
:1015B90008DBF91216181215F6901A2822E493F688
:1015C90022E6438F01538FFD75EF0275B7A575B7F5
:1015D900F1F0538FFE22438F02438F0175EF02759D
:1015E900B7A575B7F1901A0DF0538FFC22901A0D1B
:1015F900745AB1CB901A0E74A5B1CB227A3079D036
:101609007820901A40B1C6E520F709A3DAF7227AC3
:101619003079D0901A40E7B1CB09A3DAF922AB743B
:10162900A875BB01027984BB02027985BB030279E3
:1016390086BB04027992BB05027987BB060279A3AE
:10164900BB0702799CBB08027988BB09027989E842
:10165900F7227C0512059CDCFB22C2AF1205AC12F5
:1016690005B31205BA1205C112058D1205AC120592
:10167900B31205BA1205C112058D1205AC1205B3D4
:101689001205BA1205C1D2AF22C2AF1205C11205A5
:10169900BA1205B31205AC12058D1205C11205BAAD
:1016A9001205B31205AC12058D1205C11205BA1245
:1016B90005B31205ACD2AF22AE74AF75C2AF120535
:1016C900AC1205AC1205AC12058DDEF21205C11281
:1016D900058DDFF8D2AF22D163D15BD15B7574017F
:1016E900757501757600D1C17C05AD5C12059CC389
:1016F900ED955C70F5C3E55C9401400AC3E55C9423
:10170900FF403202171CD127B184D163C2AF75EFF4
:1017190012D15BDCD50576C3E5769403500280C609
:10172900D15B0575E5741490009F93F808C3E575BE
:1017390098500280AED15BD15B0574C3E574940AFD
:101749005002809C120EADB184C2AF75EF12D15B0D
:0319FD00020FFDD9
:101A00000E0615FFFFFFFF0304080101015AA5019F
:101A1000FFFFFFFFFF03FFFFFF25D0FAFA04FF01DE
:091A2000007AFF0101000300FF40
:101A400023506F6C61726973546472363041232085
:101A500023424C48454C4923463333302320202031
:101A60002020202020202020202020202020202076
:101C0000C2AFC2D353D9BF7581C043B20343FF8073
:101C1000752438752503B1C975EF0275E24043F1AB
:101C20008053A47F75D4FFD2877DFA780379E67C50
:101C300010752200752300901DD67B0675249875BB
:101C400025013087028142208708D8FBD9F9DCF7CB
:101C500081B4308708D8FBD9F9DCF781B4B189E4C5
:101C600093A3C39A6004DDC381B4DBDBB17B600264
:101C7000812B7B08E493FAA3B15CDBF87A30B15C8A
:101C8000752200752300B17BEAFCEBFDC3ED94FEE9
:101C9000400EB17B8A278B28ED30E0048A828B834B
:101CA000B17B7AC270D8C3ED94FE601350CEBD00F4
:101CB00025EC60097520007521FF0200008100A855
:101CC00027A9280809D804D90281D3B17FEA89AAB3
:101CD000F281C50D81A0C3ED94035049EDA2E092BD
:101CE000007AC5C3E5829400E583941C50902000DF
:101CF00010438F02438F0175B7A575B7F1F030001F
:101D00001FA827A9280809438F01538FFDD804D99C
:101D100002A12089AAE275B7A575B7F1F0A3A10DBC
:101D2000538FFC817C7AC1BD030CE493A3FAB140CC
:101D3000DCF8B138817C817EAA22AB23B15CEBFA5E
:101D4000EA6222752608C3E52313F523E52213F57D
:101D50002250066323A0632201D526EAB1C9B1C986
:101D600075260AEAF4200102D287300102C287B147
:101D7000C9C3134002C201D526EB22B17FEAFB2082
:101D80008702A17F308702A184752608AE24AF2583
:101D9000C3EF13FFEE13FEB1CDB1C9C3EA13308711
:101DA000024480FA30E703632201C3E52313F523DD
:101DB000E52213F52250066323A0632201D526D91C
:101DC000E52265236523F52222AE24AF250E0FDE22
:101DD000FEDFFCD20122424C48656C693437316326
:041DE000F3300601D5
:00000001FF
